:100000000C9456000C9460000C9460000C946000FA
:100010000C9460000C9460000C9460000C946000E0
:100020000C9460000C9460000C9460000C946000D0
:100030000C9460000C9460000C9460000C946000C0
:100040000C9460000C9460000C9460000C946000B0
:100050000C9460000C9460000C9460000C946000A0
:100060000C9460000C9460000C9460000C94600090
:100070000C9460000C9460000C9460000C94600080
:100080000C9460000C9460000C9460000C94600070
:100090000C9460000C9460000C9460000C94600060
:1000A0000C9460000C9460000C94600011241FBE3E
:1000B000CFEFCDBFD7E2DEBF0E9462000C947C0080
:1000C0000C94000088E18093550080E180935000FB
:1000D0008091510084FFFCCF88ED84BF84E0809341
:1000E000400080E180BB81BB81E084BB92E086B3AD
:0C00F0008927869585BBFBCFF894FFCFD5
:00000001FF
